:0A00060000308A001C2800002230A0
:100010008400000803191B280130F800F701F70BD2
:100020000F28F80B0E284A30F700F70B15280000B0
:100030000000800B0C28003484011F3083058316D8
:100040001F08C0399F009B01073083129F001E309C
:10005000831685008601831286010510860A00300A
:1000600085180130013C031D472805140430A10008
:10007000FA30A2000720A10B382805100430A10097
:10008000FA30A2000720A10B40282F284B2814305B
:0A009000A20007202E282E2863008E
:040000008A01032846
:02400E00693F08
:00000001FF
